:020000040000FA
:02000000F328E3
:0800080008002A0782070E34EC
:10001000113411341134113411340E3404340C34CD
:1000200004340434043404340E340E3411340134F2
:100030000234043408341F340E34113401340634CD
:10004000013411340E34023406340A3412341F34AD
:10005000023402341F3410341E340134013411349C
:100060000E340E34103410340E34113411340E3476
:100070001F340134013402340234043404340E34A5
:10008000113411340E34113411340E340E34113451
:1000900011340F34013411340E3400340034003480
:1000A00000340034003400340434003404340034A8
:1000B00000340E34113411341F341134113411341E
:1000C0001F341134113411341134113411340E34FD
:1000D0001E34113411341134113411341E341134DE
:1000E00011341E34113411341E34103410341034D1
:1000F0001034103410341F34103410341C341034C5
:1001000010341F34103410341C34103410341034B4
:100110000134013401340134013411340E3411340A
:1001200010341334113411340E34113411341134A9
:10013000153413340E34113410340E3401341134A8
:100140000E34113410341034103411340E3404349D
:1001500004340434043404340E34113412341434AA
:1001600018341434123411341B341534113411344E
:100170001134113419341534133411341134113449
:100180000A340434043404341E34113411341E345B
:100190001434123411341134113411341134113433
:1001A0000A3404340A34113411341134113415343E
:1001B0001B3411341F340134023404340834103435
:1001C0001F340434043404340434043404341F3439
:1001D0001F341F341F341F341F341F34EC22FE30F1
:1001E0008D009921080083160030880008118900CD
:1001F0000E308500E0308600033081008312FF302E
:100200008D0099210608C039031D3129861E242935
:10021000C73088008901EE20890A091F0B290430A4
:10022000890046308800EE20890AC4308800EE201C
:10023000890A00308800EE20890A23308800EE20E9
:10024000890A47308800EE203E308900423088001D
:10025000EE20890AEC308800EE20890A4B308800B5
:10026000EE2095019401930192019101A8018F0163
:10027000AE01AD012D1600308900582123308D00CC
:10028000992152234F220030AE00B6210F308D004D
:10029000992178308D00A0210E308D009921762390
:1002A000C130AE00B621192329308D0099213D2996
:1002B0008F210430101C05308D0081218F2100001A
:1002C0008D0B5D29802100000510932104308D00E5
:1002D00080210514932105106D2900008D0B6829DC
:1002E0008021000005148E210430101803308D0089
:1002F00081218F2100008D0B78290C308521080089
:1003000081290D308529000000008C008C0B862986
:100310000800000000000000000008008F29051000
:10032000932105140800811B0516811F0512080082
:100330008C218F21213083218D0B982908008C215D
:100340008F21023084210730A9000F30850400304E
:100350006500AA298B21FE308507A90BAA298A21CD
:100360000E30650000008D0B9F2908008F2107309B
:100370008D00FF30AA003F30B423881DAE173E30F9
:10038000B4232E1C880E080D0F39AE040F0DF03962
:10039000AE1FAE0400308900163084210430A9005D
:1003A000AA0A8E21160805209F0017080520A00024
:1003B00018080520A10019080520A2001A08052028
:1003C000A3001B080520A4001C080520A5001D088B
:1003D0000520A6001E080520A700073085218A21D8
:1003E0008F218A218C212E080E3985040030881D2A
:1003F00065002E1F8C21AE1AFF29FE2900002E1E3B
:10040000012A1F088600860D860D860D860D860141
:1004100020088600860D860D860D860D8601210832
:100420008600860D860D860D860D860122088600C3
:10043000860D860D860D860D860123088600860DA5
:10044000860D860D860D860124088600860D860D94
:10045000860D860D860125088600860D860D860D83
:10046000860D860126088600860D860D860D860D72
:10047000860127088600860D860D860D860D86016D
:100480002E1B8C21AE1E462A452A00002E1A482A11
:100490000E306500A90BEF298D0BCE2908008E21A7
:1004A000861AAD01861EAD142D143F30B423582A90
:1004B000592A2D1A632AAD19C82A2D19962AAD1862
:1004C000982A0000642A8B210E23031D702A060837
:1004D000C03903198D2A081B8813881B762A812AA4
:1004E000AD01AB01AF01113083210800061B940A56
:1004F000861B920A950152300E1B8E000D3085210D
:1005000008003E30B423861B880E8811880A861B9B
:10051000880EEC2206308421C42A80300813880615
:100520000E1B0817EC220B308321C42A3530A8009B
:100530008F0108302D1DAF000E23031DAD2A0608C4
:10054000C0390319B02AF622072316302F0784007A
:100550002C08800003308321080005308421A42A60
:1005600028082F0789003D3A031DA80A031DAF0A7A
:10057000AB012C088800E03A0319AF010319AD0D57
:10058000031DEC2207308321E0308D00992153298F
:100590000808AB000E230319D02A14308421080068
:1005A000061FE62A8F01AB0D2B10AB192B14103050
:1005B000AB19AB07AB112B1AAB15F03088052B0824
:1005C0000F398804EC220A308521C42A203088069D
:1005D000EC220E308421C42A831608155530890078
:1005E000AA3089008814081183120800861BAB0A00
:1005F000061BAB032B08FF3A27300319AB002B086F
:10060000283A0319AB0153300E1B8E00080003304B
:100610008A002B08BA23AC008A0108000609C039F9
:100620002A3003198E008E0A32300E1B5A300E0605
:1006300008008E21900ACE3010070318900103188D
:10064000950A03180000C430150703189501031814
:10065000940AF6301407031894010318930AFA3029
:100660001307031893010318920AF63012070318B0
:1006700092010318910A120811180A3E9118FC3EC3
:1006800003189201031891013F30B4230030890010
:1006900003301518881A04308316810083120E3037
:1006A000852108008E213F30B423AE0007398F0723
:1006B0000F08C83E03188F010318A80A5F2B2808EB
:1006C000CA3EF8300319A8002808B423473AF83086
:1006D0000319A800280889001630840014308421EA
:1006E000A223A22B0530832135306B2B8E213F3086
:1006F000B423081B7E2B881B802B722B1519722BA1
:1007000046309600970098009E00031011089B2326
:10071000990012089B239A004B30151846309B0015
:1007200013089B239C0014089B239D000A308321FF
:1007300002308D0099298C008C0D8C0D8C078C0754
:100740000C0708008E21AA23AA23AA23AA23AA23DE
:1007500089210800B523091B46308000840A473AE6
:1007600003190917890A08008900831608148312DF
:10077000080808008207E034523467349934613441
:1007800074347A34873456349F348134A6346E34CA
:10079000AC34B13400346A348D34BD349334D9343C
:1007A0005A34C434CC34C734B634D3344634003429
:1007B00007340E3415341C3423342A34313438349D
:0607C0003F344B344734C6
:02400E00F23F7F
:104200004B3493340034BD34BD34B63446347A3440
:104210000034BD34463467345A34873493344634DA
:104220009F34B1344634C434C734C73446344B3475
:104230004634873400340034613446346E345A34A2
:104240009934A6344634CC349F34D9345634463469
:10425000D93456349F3493344634C4340034233430
:10426000463446346734B6344734463446349F3493
:10427000CC340E34A6348734563446344200EC0035
:00000001FF
